:030000000219FDE5
:03000B000200AA46
:03002B0002019936
:03005B0002034C51
:0300730002033253
:1000800002030406080C10182030406080040608A3
:100090000C10182030406080A0C000070F1F3F0DDB
:1000A0000D04050D050305030302C2AF306308C24A
:1000B00063857C8AD2AF32C0D0C0E0206227E525BC
:1000C0006002E473E525F4C3334009758A00D26306
:1000D000F57C01D6F58A758B00758D00D262D0E073
:1000E000D0D0D2AF32C3E526334009758A00D2633F
:1000F000F57C01F6F58AC262E526F4603B306803C0
:10010000207213758B00758D00D0E0D0D0D293D2C1
:1001100097D295D2AF32D293D297D295206E0C203F
:1001200066097410D5E0FDE57E4290758B00758DF3
:1001300000D0E0D0D0D2AF32758A00D263757C0097
:10014000C28DD262212B01C4306805206602C293A1
:1001500001C4306805206602C29501C430680520DC
:100160006602C29701C4C29230680A2066077416FC
:10017000D5E0FDC29301C4C29430680A20660774BA
:1001800016D5E0FDC29501C4C29630680A20660704
:100190007416D5E0FDC29701C4C2AFC2AD53E6EFFD
:1001A000C0D0C0E0D2D3D2AFE57D6009E57A60056A
:1001B000757A0041DF757A01C2CEE52A60072074A6
:1001C00049152A410A7800790020742EE580307E96
:1001D00001F430E50278FF53DACF207E0343DA20C2
:1001E000307E0343DA10C2D8C271E580307E01F45C
:1001F00030E50279FFC3E89970CB306103752A18A6
:10020000207403752A18885FD27020740DE52B6066
:1002100004152B411A43DA01C2D82070024178A894
:100220005F206102C2702074367982B70431C3E85E
:1002300094F0400374F0F8E8C4540F28F87984B7B8
:100240000302415FC313C3138721200802C3132095
:100250000A06C3C898F8415F28F8500374FFF8886D
:1002600022E52D54066011E533C313C3132406257C
:1002700022F52250037522FF7882B6045985222484
:10028000A824C3E52495644002A864C3E8956640A9
:1002900002A8668825E569700241C9C3E8AA699A7F
:1002A0005003E8FAE4F9EAC333FBE56BF45B294059
:1002B0000D256AF8E56A6002156A400B41C90AC358
:1002C000E56A9A5002056A78FF8826C26EC3E52661
:1002D00094F84002D26EC3E52594404002D26420D7
:1002E000CF0AD0E0D0D043E610D2AD32C2CF053A2B
:1002F000E57D6009E57B6005757B006128757B0104
:100300007801E52A6005307402152AC3E55F94017F
:1003100040057562006128756300756C00E5622414
:1003200001F56250037562FFD0E0D0D043E610D2F1
:10033000AD32C2AFC0D053E67FC260759100855622
:1003400094855795759104D0D0D2AF32C2AF53E6A1
:10035000EFC2ADC0D0C0E0C0F0D2D3D2AFA8FBA9ED
:10036000FCE57D6007C3E913F9E813F8C2D83071E2
:100370000261BE53DACF207E0343DA10307E03439E
:10038000DA20D271E580307E01F420E502619588A3
:10039000278928A1EB53DACF207E0343DA20307E71
:1003A0000343DA10C2D8C271307402A1D77800E5D5
:1003B00080307E01F430E502A1D7885FA1BF53DA17
:1003C000CF207E0343DA20307E0343DA10C271204F
:1003D0006102819753DACF207E0343DA10307E0327
:1003E00043DA20C2D8D271885A895BC3E89558F89D
:1003F000E99559F97B007E087A00C3E8948CE9946A
:10040000005005755E008189882178A2E6A82160E8
:1004100055C3E894C8E994005008E4D2E4FB7A0A92
:100420008164C3E89468E994015008E4D2E3FB7A5C
:100430000F8164C3E894D0E994025008E4D2E2FB4F
:100440007A1E8164C3E894A0E994055008E4D2E1DF
:10045000FB7A3C8164C3E89498E994085008E4D29C
:10046000E0FB7A787E00C3E8955CFCE9955DFD30A1
:0F047000E70AECF42401FCEDF43400FD755E00A6
:10047F00C3EC9AED9E5003755E01885C895D855AC9
:10048F0058855B597802A1BFC3E89527F8E99528ED
:10049F00F9307C02A1A3307B02A1A3307A02A19C88
:1004AF0020750281BAE9FDE8FC81D9E9C313F9E8A7
:1004BF0013F8307902A19CE9C313F9E813F83078E7
:1004CF0002A19CE9C313FDE813FC20612CC3EC943B
:1004DF001CED9402400281F0ED701EC3EC94C850E5
:1004EF00180529E52970021529C3E529940A500238
:1004FF00A1D7755F00D270A1D7E5296002152978C1
:10050F0088E6F97400207F087896B90302789EE692
:10051F0024FAFEE43400FFC3EC9EFCED9FFD92082D
:10052F00B90310A2085007207609D276A14230767F
:10053F0002C276A2085016B9030DECF42401FCEDAB
:10054F00F43400FD02055C78007900A1A3B903150E
:10055F00EC33FCED33FDC3EC940AFCED9400FD503D
:10056F00047C007D00C3EC94FFED9400400678FFFF
:10057F007900A1A3EC8575F0A4C5F0A2F733F87943
:10058F000040030205BF78FF79000205BFE9C313DE
:10059F00F9E813F8307C0EE9600278FFC3E81338EE
:1005AF00F8E43400F9C3E894FFE99400400278FFBF
:1005BF00885FD270206102A1D7741FF4552F4BF5BD
:1005CF002FC274EB7002D274752A18307403752A17
:1005DF000A306102A1EB20740353DAFE2074037515
:1005EF002B06D0F0D0E0D0D0D2AD43E61032790157
:1005FF0002061B790302061B790A02061B791E02EB
:10060F00061B796402061B79C802061B7817E4D50E
:10061F00E0FDD8FAD9F6227A147B780206427A10D6
:10062F007B8C0206427A0D7BB40206427A0B7BC8A2
:10063F000206427902B27DE4C294D5E0FDC295D59F
:10064F00E0FDD295D5E0FDD294D5E0FDC293E576DD
:10065F00D5E0FDD2937496D5E0FDD9D9EAF8D5E06F
:10066F00FDD8FBDBCEC29422C37C007D0075F00069
:10067F0005F0EA33FAEB33FB50F6EB13FBEA13FA10
:10068F00C3E9FFE8FEE89AF8E99BF95004EFF9EEA9
:10069F00F8B3EC33FCED33FDD5F0DFEDF9ECF822D8
:1006AF00E889F08A20D2D4F8A9F07B0030F70B7BD1
:1006BF00FFF42401F8E9F43400F9E88520F0A4AD43
:1006CF00F0F8E98520F0A4AFF0FEED2EF974003FAD
:1006DF00FA7C04C3EA13FAE913F9E813F8DCF48B94
:1006EF00F030F70AE8F42401F8E9F43400F9E88966
:1006FF00F0C2D4F8A9F0227882B60403020761C3CE
:10070F00E55F9401400302072B852224E4F545F5AC
:10071F0046F547F548F549C26D0207617882E6FC58
:10072F00D26DE522F523783879C7AA40AB41C3EBE8
:10073F0013FBEA13FAEC146013C3EB13FBEA13FA7F
:10074F00EC14146007C3EB13FBEA13FAD177884557
:10075F00894622C3E5459523F8E5469400F9500CE8
:10076F00C3E89480E994FF4016020792C3E8947F90
:10077F00E994005003020792787F7900020792787C
:10078F008079FF884A894B22E54A2547F8E54B35A2
:10079F0048F9854B20E4300701F43549FA30E70971
:1007AF00C3EA94F040150207D0C3EA940F50030236
:1007BF0007D078FF79FF7A0F0207D0780079007A97
:1007CF00F0C3E5249564500AC374019524500B02BD
:1007DF0007EEE54B20E70E0207EEE54B30E7068804
:1007EF004789488A492278A4E6FAC3E54A33F8E5EF
:1007FF004B33F91206AFE930E70BC3E89480E99465
:10080F00FF40130129C3E8947FE9940050020129A6
:10081F00787F79000129788079FFE820E715C3E513
:10082F002398F84009C3E894014003020850780167
:10083F00020850E8F424012523F8400302085078F9
:10084F00FF884C2278A5E6FAA848A9491206AFE915
:10085F0030E70CC3E89401E994FF4016020885C302
:0F086F00E894FFE99400500302088578FF7900B0
:10087E00020885780179FFE920E715C3E54C98F861
:10088E004009C3E8940140030208AC78010208ACA9
:10089E00E8F42401254CF840030208AC78FF8824C4
:1008AE002278FFC26420693D206A12D264C3E541FA
:1008BE00940A4009C3E52594405002C26479A1E729
:1008CE006023E541601F74FF8541F0848539F03067
:1008DE006A0375F005A4F8C5F0600278FFC3E895C9
:1008EE00675002A867886622C3E54094C8E5419424
:1008FE0000E5665003142107046002F56622020922
:10090E000F2275E890227883E6FFE5E820ECF7A841
:10091E00BDA9BE0573C3E57394084052757300E913
:10092E00FA79A0E76044EA7007E574601B02094A91
:10093E00C3E895746010E5745006600C14020956F5
:10094E000460F9020956E574F574C39472401B7580
:10095E0064C0C394044013756480C39404400B7543
:10096E006440C39404400375640075BB0822E564BB
:10097E002410500274FFF5647982B7040221A3C3D8
:10098E00A864E524985002A824C3E895664002A8FE
:10099E006688258826E573B4070375BB102274326A
:1009AE0079A687F0A4C5F0A2F733F8C3E8956440A2
:1009BE0002A86488228824882588268867227540A4
:1009CE00007541F022C2AF75C820A8CCA9CDAA3AB5
:1009DE0030CF010A75C824D2AFC3EA13FAE913F96E
:1009EE00E813F8AB3BAC3C883B893CC3E89BF8E989
:1009FE009C20690A547FF930670241F64153AD3DA0
:100A0E008A3DF9EA9D547FFA600478FF79FFAE3E85
:100A1E00AF3F8B3E8C3FC3EC9FFCC3E99CF542A8D5
:100A2E003BA93CC3E89EF8E99FF9C3E54113FBE5FA
:100A3E004013FAE82AF540E93BF54150067540FFB0
:100A4E007541FF419DAA40AB41AC40AD417E047F54
:100A5E0002C3EB940440021E1FC3EB940840021E17
:100A6E001FC3ED13FDEC13FCDEF7C3EA9CFAEB9DFE
:100A7E00FBEF6009C3E913F9E813F8DFF7EA28FA88
:100A8E00EB39FB8A408B4150067BFF8B408B41C379
:100A9E00EB94025002D2673069047F0341C878920A
:100AAE00E6FFC3E537948240110FC3E53794A040AB
:100ABE00010FC3EF940640027F057E03E541C45447
:100ACE000FF9E541C454F0F8E540C4540F28F8C3BB
:100ADE00E89EFAE99400FB4009C3EA9402EB940005
:100AEE0050047A02E4FB6142AA40AB41EBC4FEEA39
:100AFE00C4540F4EFCC3EA9CFAEB9400FBC3E813FC
:100B0E00C313F8EA28FAEB3400FB8A408B41C3EB9F
:100B1E0094024002C2677803EBC4FE7B00EAC45421
:100B2E000F4EFAC3EA98FA4005C3940250027A02B5
:100B3E007892E6FF3060026142855256855357D255
:100B4E006043E680C3E49AF8E49BF9C3E833F8E91E
:100B5E0033F930670261E3E8FAE9FBD3E913FDE804
:100B6E0013FC88528953C3EF94036038EF20E00DD5
:100B7E00E82CF8E93DF9ECFAEDFB020B9EE828F8BB
:100B8E00E939F9C3E82402F8E93400F97AFE7BFF6B
:100B9E00C3EF9403400E8A548B55884E894F8C5068
:100BAE008D518117885489558A4E8B4F8C508D519B
:100BBE00306920C3E53394034019E542A2E713F8E8
:100BCE00E555F4240138400B20E7087554FFF42452
:100BDE0001F5558117E8FAD3E813FC8852C3EF9458
:100BEE00036020EF20E007E82CF8ECFA8103E828F8
:100BFE002402F87AFEC3EF940340088A54884E8C80
:100C0E0050811788548A4E8C50E56BC33350026462
:100C1E006BF56B3060028121753404D26043E6803F
:100C2E00E52D5406601FA840A941C2AF53E67F755B
:100C3E009100C3E498F594E499F595759104D2600A
:100C4E0043E680D2AF22D265754400752000306B2A
:100C5E0003752040020C73D2657544007520403038
:0E0C6E006B03752000D2AF7801206722E52DC0
:100C7C0054066002C265C3E54194054013780294A2
:100C8C000540087803940540027806306902780A1A
:100C9C00206019E544601530690AC3E533940340BC
:100CAC0003D53406D2AFD26CA1559129D2AF000036
:100CBC00C2AF20672AE541C3FB940F40027B0FEBC8
:100CCC00240530730123306A02742820620123F951
:100CDC003069027982E58D13E58B13C39940B10518
:100CEC0044E59B5440B52002A13F30690A08C3E893
:100CFC00940A400108819C2065028173C26553E609
:100D0C007F7591003067107594007595FC75910492
:100D1C00D26043E6808173AE40AF41C3EE33FEEF49
:100D2C0033FF50047EFF7FFFC3E49EF594E49FF5F0
:100D3C0095A119C3E5339402500281733065028189
:100D4C0073D802A153819CC26C53E67F75910085C8
:100D5C005494855595759104854E56854F57D260A0
:100D6C0043E680D2AFE52D54066008206A020533B5
:100D7C00020D8F306C0D206B0A20650715811581D3
:100D8C000216082278003064053065027801E537D8
:100D9C0075F007A4F9E5F028F5F0E9A2F013A2F13B
:100DAC0013A2F213F537C394785003753778C3E563
:100DBC003795384008D266D293D297D295306002DC
:100DCC00A1C9855056855157D26043E68022207DBB
:100DDC0011C2AF754302C294D292D2AF759F40023A
:100DEC000FA9C2AF754302C294D296D2AF759F4081
:100DFC00020FA9307243207D20C2AF7543039001CE
:100E0C0077757E10D297C296306204C295C11DD2FE
:100E1C0094D2AF759F41020FA9C2AF7543039001E5
:100E2C0077757E10D293C292306204C295C13DD2C6
:100E3C0094D2AF759F43020FA9207D17C2AF7543A3
:100E4C0003900152D297306202C295D2AF759F4186
:100E5C00020FA9C2AF754303900152D293306202C4
:100E6C00C295D2AF759F43020FA9207D11C2AF75F9
:100E7C004304C292D296D2AF759F43020FA9C2AF60
:100E8C00754304C296D292D2AF759F41020FA9301E
:100E9C007243207D20C2AF754305900166757E04B8
:100EAC00D295C294306204C293C1B9D292D2AF75BA
:100EBC009F40020FA9C2AF754305900188757E4013
:100ECC00D295C294306204C297C1D9D296D2AF7572
:100EDC009F40020FA9207D17C2AF754305900148B2
:100EEC00D295306202C293D2AF759F40020FA9C255
:100EFC00AF75430590015CD2953062EBC297D2AFCF
:100F0C00759F40020FA9207D11C2AF754306C29692
:100F1C00D294D2AF759F41020FA9C2AF754306C2DE
:100F2C0092D294D2AF759F43020FA9307242207DAA
:100F3C0020C2AF754301900188757E40D293C29256
:100F4C00306204C297E155D296D2AF759F43020F1F
:100F5C00A9C2AF754301900166757E04D297C29603
:100F6C00306204C293E175D292D2AF759F41E1A970
:100F7C00207D16C2AF75430190015CD293306202A2
:100F8C00C297D2AF759F43E1A9C2AF7543019001DF
:100F9C0048D297306202C293D2AF759F41C266228B
:100FAC00900146757E00D293D297D295C292C2968A
:100FBC00C294C26222788076090876090876040801
:100FCC0076FF0876030876FF08760B08760308761A
:100FDC0001087601788C76010876FF0876FF087692
:100FEC00FF0876FF0876FF0876030876FF0876FF81
:100FFC000876FF0876250876D008762808765008FB
:10100C0076040876FF08760208760008767A087669
:10101C00FF087601087601087600087603227887A7
:10102C00E6FFC272BF0302D2727888E6C3940360F3
:10103C0008C27DE630E102D27DC27E7889E630E1DD
:10104C0002D27EC3EF94026008758E01D273021037
:10105C0062758E00C273227880E6149000809378BB
:0F106C00A4F67881E6149000809378A5F6788634
:10107B00E61490008D9378A6F6789CE67538FF758C
:10108B00390CB402067538A075390AB403067538E5
:10109B008275390578A3E61490009A93F569120FBF
:1010AB00AC22227896E6FA7897E6FB7888E6B403CA
:1010BB0005C3EB940EFB307F047A007BFFC3EB9AE6
:1010CB00FCC3948250027C827575000575EC8575A6
:1010DB00F0A4C3E5F0947D40F222D27F11AE12064C
:1010EB000C7A007B007C10120602E55F2AFA740072
:1010FB003BFBDCF37C04C3EB13FBEA13FADCF7FEDC
:10110B00C27F11AE22E5EF20E6037520000520908B
:10111B003FFFE520146006901FFF146000930460EE
:10112B000375EF1253D9BF7581C043FF801205FDC4
:10113B0075EF0243B203E5B3240420E70DF521E577
:10114B00E320E0068521B343E301120FAC7580FF6A
:10115B0075A40075F13075D4DF7590AB75A5FC7572
:10116B00F2FC75D50175A60175E241E4F8F6D8FDE0
:10117B00756B01120FC11216527898867675300175
:10118B00C2AF12061612062612060C12062D1206F6
:10119B000C12063412060CC2AF78FA79FA308507B6
:1011AB00D9FBD8F7021C00112A116311AD11AE78CF
:1011BB00988676120FAC75A90075B680757D007593
:1011CB00885075891275C82475910475D84075A817
:1011DB002275B80275E690759B80759D0075D10ED2
:1011EB0075BCC075BB0875BA1175E8801205FDD2C8
:1011FB00AF12090C53DACF207E0343DA20307E0383
:10120B0043DA1043DA01C2D8C271120616D2617BDF
:10121B00037A0CE55E70077A0CDB030211A212064F
:10122B000C2070030211A2C270E55FC3940240E16F
:10123B00E52F541F856160F561B560D5DAD5C261C4
:10124B0053DACF207E0343DA20307E0343DA10C219
:10125B00D8C27178A2E67008D274E52F54E0F52F4E
:10126B00C275752900120611307409C3E529940A59
:10127B004002D27512060278023074027800C3E580
:10128B005F9840F0C2AF120626120626120626D22F
:10129B00AF120616754D007888E6B4030261801212
:1012AB000602788CE6C394015003021380E530C329
:1012BB0094015003021380207435C3E55F94FF50F3
:1012CB0003021380C2AF12063BD2AF120611C3E565
:1012DB005F940150EFC2AF120626120607120626C4
:1012EB00D2AF120611C3E55F94FF40E90217FA7FF4
:1012FB0002D27F11AE120611C2AFC27F11AEAE5F2A
:10130B00C3E55F947FD2AF40761205FDC2AF1206E4
:10131B003BD2AFDFDC11E5C3EE94057897F61206EE
:10132B001612169412177D7F0AD27F11AE12061178
:10133B00C2AFC27F11AEAE5FC3E55F947FD2AF5039
:10134B00E61205FDC2AF120626120607120626D2BA
:10135B00AFDFD611E5EE24057896F61206161216B7
:10136B00941217AC12061111AEC3E55F94FF500235
:10137B0041C20217FAC3E55F954D4003855F4D12DD
:10138B00061178017988E7B403027805C3E55F9805
:10139B00400241A2C2AF12063B12063B12063BD2E1
:1013AB00AF120616753000E4F531F5320531E53133
:1013BB00F470390532789AE6781914601278321481
:1013CB00600D787D14600878FA146003753200C3E1
:1013DB00E53298401715327531B478998676C2AFDD
:1013EB0012063BD2AF78988676120611120607E5E5
:1013FB002A700530740221A278012074027806C38A
:10140B00E55F9840A77888E6C39403600312061142
:10141B00E52A70030211A2C2AF120FACE4F522F55C
:10142B0023F524F525F526F56AD2AF7885E6C33387
:10143B00F568E4F545F546F547F548F549F573F5D7
:10144B002CF52DF53775730875BB101205FD1209B8
:10145B0010E5E820ECFBA8BDA9BEE97001F8887483
:0F146B0012091475730875BB107887E6FE7602B8
:10147A00112A7887EEF6C2AF7564FF1209AC85228D
:10148A0064852265852266D2AF75220175240175AD
:10149A00250175260185636C756D0175B69075A970
:1014AA0003757D017888E6B40307C27D307602D2DF
:1014BA007DD268D269753300120F12120F371209E2
:1014CA00CC1209D31209CC1209D31209CC0214E6A0
:1014DA00C2AF112AD2AF75730075BB08120C651220
:1014EA000706120D90120DDA1209D3120C54306D40
:1014FA00031207622067031208AF3067031208F667
:10150A00120D90120DFF1209D3120C65306D0312E1
:10151A000797120D90120E761209D3120C54306DE1
:10152A00031207F5120D90120E9B1209D3120C65C5
:10153A00306D03120853120D90120F121209D312B2
:10154A000910120C54120D90120F371209141209B5
:10155A00D3306935206B3285676485676585636C2E
:10156A00756D0179187A0CC3E53399400FC269D2B7
:10157A006A8A35856764856766021593C3E55F9451
:10158A000140030214E6021610306A1B206B18E5AC
:10159A0035147004C26A81DAF535C3E55F940140F7
:1015AA00030214E6021610753600C3E56278FA984B
:1015BA005054307404E52A604D7888E6B403172045
:1015CA007D05207607A1E0307602A1E0206B07D2E4
:1015DA006B856764A12578F0306B05856764782090
:1015EA00C3E54198500281E6306B1BC26BC27D3065
:1015FA007602D27DD26A75351285676481E6053630
:10160A00E55F6002C113753600C2AF120FAC78876E
:10161A00E6FE7602112A7887EEF6E4F522F523F53E
:10162A0024F525F526F568C26875A90075B6807592
:10163A007D00D2AF1205FD120FAC307409C3E53636
:10164A009405400221A261B2901A0D78201216D692
:10165A00E520B4550CA31216D6E520B4AA03021647
:10166A0074120FC1121694021693901A0378807B93
:10167A000A1216D6A308DBF9901A0F788C7B181277
:10168A0016D6A308DBF9901A2722C2AF1217151231
:10169A0016EF901A00740E1216DBA374041216DBEE
:1016AA00A374141216DB901A0378807B0A1216DAD6
:1016BA00A308DBF9901A0F788C7B181216DAA308A4
:1016CA00DBF9121728121706901A2722E493F6223A
:1016DA00E6438F01538FFD75EF0275B7A575B7F114
:1016EA00F0538FFE22438F02438F0175EF0275B7C5
:1016FA00A575B7F1901A0DF0538FFC22901A0D744C
:10170A0055D1DB901A0E74AAD1DB227A3079D078BF
:10171A0020901A40D1D6E520F709A3DAF7227A30C9
:10172A0079D0901A40E7D1DB09A3DAF922AB77A87E
:10173A0078BB01027980BB02027981BB03027982FC
:10174A00BB04027984BB05027986BB06027992BB87
:10175A0007027987BB080279A3BB0902799CBB0AF5
:10176A00027988BB0B027989E8F7227C05120616F2
:10177A00DCFB22C2AF12062612062D12063412060E
:10178A003B12060712062612062D12063412063BD3
:10179A0012060712062612062D12063412063BD22C
:1017AA00AF22C2AF12063B12063412062D120626CB
:1017BA0012060712063B12063412062D12062612CC
:1017CA00060712063B12063412062D120626D2AF5F
:1017DA0022AE77AF78C2AF12062612062612062666
:1017EA00120607DEF212063B120607DFF8D2AF2214
:1017FA00F17DF175121775757701757801757900A4
:10180A001217DB7C05AD5F120616C3ED955F70F506
:10181A00C3E55F9401400AC3E55F94FF40370218AD
:10182A003C12173712169412177DC2AF75EF1212B7
:10183A001775DCD10579C3E5799403500280C1128A
:10184A0017750578E5771490009F93F808C3E57833
:10185A0098500280A81217751217750577C3E57795
:0E186A00940C50028094120FC1121694C2AF5B
:0618780075EF1212177556
:0319FD00021110C4
:101A00000E0414090904FF03FF0B03010155AA0189
:101A1000FFFFFFFFFF03FFFFFF25D0285004FF0259
:081A2000007AFF01010003FF41
:101A40002358526F746F72313041232020202020A0
:101A500023424C48454C492346333930232020202B
:101A60002020202020202020202020202020202076
:101C0000C2AFC2D353D9BF7581C043B20343FF8073
:101C1000752438752503B1C975EF0275E24043F1AB
:101C20002053A4DF75D400D2857DFA780379E67C51
:101C300010752200752300901DD67B0675249875BB
:101C400025013085028142208508D8FBD9F9DCF7CF
:101C500081B4308508D8FBD9F9DCF781B4B189E4C7
:101C600093A3C39A6004DDC381B4DBDBB17B600264
:101C7000812B7B08E493FAA3B15CDBF87A30B15C8A
:101C8000752200752300B17BEAFCEBFDC3ED94FEE9
:101C9000400EB17B8A278B28ED30E0048A828B834B
:101CA000B17B7AC270D8C3ED94FE601350CEBD00F4
:101CB00025EC60097520007521FF0200008100A855
:101CC00027A9280809D804D90281D3B17FEA89AAB3
:101CD000F281C50D81A0C3ED94035049EDA2E092BD
:101CE000007AC5C3E5829400E583941C50902000DF
:101CF00010438F02438F0175B7A575B7F1F030001F
:101D00001FA827A9280809438F01538FFDD804D99C
:101D100002A12089AAE275B7A575B7F1F0A3A10DBC
:101D2000538FFC817C7AC1BD030CE493A3FAB140CC
:101D3000DCF8B138817C817EAA22AB23B15CEBFA5E
:101D4000EA6222752608C3E52313F523E52213F57D
:101D50002250066323A0632201D526EAB1C9B1C986
:101D600075260AEAF4200102D285300102C285B14B
:101D7000C9C3134002C201D526EB22B17FEAFB2082
:101D80008502A17F308502A184752608AE24AF2587
:101D9000C3EF13FFEE13FEB1CDB1C9C3EA13308513
:101DA000024480FA30E703632201C3E52313F523DD
:101DB000E52213F52250066323A0632201D526D91C
:101DC000E52265236523F52222AE24AF250E0FDE22
:101DD000FEDFFCD20122424C48656C693437316326
:041DE000F390060175
:00000001FF
